:100000000C94A8040C94E0040C94E0040C94E00418
:100010000C94E0040C94E0040C94E0040C94E004D0
:100020000C94E0040C94E0040C94DA220C94AC23BD
:100030000C942E1D0C94E0040C94E0040C94E00449
:100040000C94E0040C94E0040C94E0040C94E004A0
:100050000C94E0040C94B61D0C94E0040C94E004A1
:100060000C94E0040C94E0040C94E0040C94E00480
:100070000C94E0040C94E0040C94E0040C94E00470
:100080000C94E0040C94E0040C94E0040C94E00460
:100090000C94E0040C94E0040C94E0040C94E00450
:1000A0000C94E0040C94E0040C94E004B509B50948
:1000B000E109E109490A740B740B740B670A000B20
:1000C000110B110B192440243825402438258C2489
:1000D000AF2438250625152568747470733A2F2FC0
:1000E000716D6B2E666D2F01012800514D4B2069FB
:1000F00073207468652062657374207468696E6724
:100100002065766572210029003A003B003C003DE5
:10011000003E003F004000410042004300440045D3
:100120000046004C004A004D004B004E0035001EBA
:10013000001F0020002100220023002400250026AB
:100140000027002D002E0000002A00530054005507
:100150000056002B00000014001A000800150017BC
:10016000001C0018000C00120013002F00300000CB
:10017000005F00600061000000390000000400160C
:1001800000070009000A000B000D000E000F0033ED
:10019000003400320028005C005D005E005700E182
:1001A0000031001D001B00060019000500110010A1
:1001B000003600370038000000E500520059005AB0
:1001C000005B000000E000E300E20000000000002F
:1001D000002C000000000000000000E600E40050D9
:1001E0000051004F006200630058004445425547EB
:1001F0003A2064697361626C65642E0A004445426A
:1002000055473A20656E61626C65642E0A000000F5
:100210000000000000002A2B280000000000000061
:1002200000000000000000000029000000002C1E5B
:100230003420212224342627252E362D3738271E18
:100240001F202122232425263333362E37381F043E
:1002500005060708090A0B0C0D0E0F1011121314D6
:1002600015161718191A1B1C1D2F3130232D350494
:1002700005060708090A0B0C0D0E0F1011121314B6
:1002800015161718191A1B1C1D2F3130354C00007C
:10029000000000000000000000000000000000005E
:1002A000000000000000000000000000000000004E
:1002B00000007E0F00D4FFFFFFC7000000780A0097
:1002C00025303258006C65645F7461736B3A2000AE
:1002D0004F6E6573686F743A206163746976653A2E
:1002E0002025640A000A00253033326C62003A206F
:1002F0000025303258000A722F63203031323334F7
:10030000353637383941424344454630313233344B
:1003100035363738394142434445460A003F0043A9
:100320003E20004C25640A000A092D205374617494
:100330007573202D0A686F73745F6B6579626F61E6
:1003400072645F6C65647328293A20253032580A3C
:100350006B6579626F6172645F70726F746F636FE7
:100360006C3A20253032580A6B6579626F6172648D
:100370005F69646C653A20253032580A74696D658E
:10038000725F72656164333228293A202530386CF7
:10039000580A000A092D2056657273696F6E202D68
:1003A0000A5649443A2030784645454428456C6C05
:1003B000696F7420506F77656C6C29205049443AFE
:1003C0002030783936393628657039362920564537
:1003D000523A203078303030310A4255494C443A54
:1003E0002020284665622032372032303232290AF6
:1003F0004F5054494F4E533A204C55464120455892
:100400005452414B455920434F4E534F4C45204386
:100410004F4D4D414E4420343039360A4743433A1C
:1004200020352E342E30204156522D4C4942433A2D
:1004300020322E302E30204156525F415243483AEE
:1004400020617672350A000A092D20436F6E736FA2
:100450006C65202D0A4553432F713A0971756974F3
:100460000A000A092D204D61676963202D0A443A6C
:10047000094465627567204D657373616765205433
:100480006F67676C650A583A094D61747269782024
:100490004465627567204D6F646520546F67676CB3
:1004A00065202D2053686F77206B657970726573B6
:1004B00073657320696E206D61747269782067724C
:1004C00069640A4B3A094B6579626F617264204432
:1004D0006562756720546F67676C65202D205368CF
:1004E0006F77206B65797072657373207265706FBA
:1004F00072740A4D3A094465627567204D6F7573D1
:100500006520546F67676C650A563A0956657273C1
:10051000696F6E0A533A095374617475730A433AEA
:1005200009416374697661746520436F6E736F6C03
:1005300065204D6F64650A46312D4631303A0953C6
:10054000776974636820746F204C6179657220301C
:100550002D392028463130203D204C30290A302DBD
:10056000393A0953776974636820746F204C617954
:10057000657220302D390A47524156453A09537762
:100580006974636820746F204C6179657220302033
:1005900028616C7465726E617465290A423A094A71
:1005A000756D7020746F20426F6F746C6F6164653D
:1005B000720A4553433A094A756D7020746F2042A0
:1005C0006F6F746C6F616465722028616C74657202
:1005D0006E617465290A453A095072696E74204546
:1005E0004550524F4D2053657474696E67730A42CB
:1005F00053504143453A09436C656172204545506B
:10060000524F4D0A006B65796D61705F636F6E6666
:1006100069672E7261773A20253032580A2E737737
:1006200061705F636F6E74726F6C5F636170736C27
:100630006F636B3A2025750A2E636170736C6F636C
:100640006B5F746F5F636F6E74726F6C3A202575A9
:100650000A2E737761705F6C63746C5F6C67756989
:100660003A2025750A2E737761705F7263746C5F30
:10067000726775693A2025750A2E737761705F6C11
:10068000616C745F6C6775693A2025750A2E737703
:1006900061705F72616C745F726775693A2025756D
:1006A0000A2E6E6F5F6775693A2025750A2E73777B
:1006B00061705F67726176655F6573633A20257567
:1006C0000A2E737761705F6261636B736C6173682C
:1006D0005F6261636B73706163653A2025750A2EF2
:1006E0006E6B726F3A2025750A0064656275675FEC
:1006F000636F6E6669672E7261773A2025303258D3
:100700000A2E656E61626C653A2025750A2E6D6150
:10071000747269783A2025750A2E6B6579626F616B
:1007200072643A2025750A2E6D6F7573653A20251F
:10073000750A006565636F6E6669673A0A64656687
:1007400061756C745F6C617965723A2025750A0079
:100750003F000A6D6F7573653A206F66660A000A7E
:100760006D6F7573653A206F6E0A000A6B6579626A
:100770006F6172643A206F66660A000A6B6579627F
:100780006F6172643A206F6E0A000A6D617472695B
:10079000783A206F66660A000A6D61747269783A69
:1007A000206F6E0A000A64656275673A206F66669C
:1007B0000A000A64656275673A206F6E0A000A0AC9
:1007C0004A756D70696E6720746F20626F6F746C0C
:1007D0006F616465722E2E2E2000433E2000436C14
:1007E000656172696E6720454550524F4D0A000A97
:1007F000002530325820006B6579626F6172645F4A
:100800007265706F72743A20005B735D005B575DB8
:10081000005B535D005B525D005B445D005B435DCC
:10082000000A03650070003900360000001C034513
:10083000006C006C0069006F007400200050006FB5
:1008400000770065006C006C0000000403090409D7
:10085000025B00030100A0FA09040000010301018A
:100860000009211101000122400007058103080051
:100870000109040100010300000009211101000128
:10088000223200070582032000010904020002034E
:100890000000000921110100012222000705830345
:1008A00020000107050303200001120100020000DF
:1008B0000008EDFE96960100010200010631FF09D5
:1008C00074A1010975150026FF00952075088102A5
:1008D0000976150026FF00952075089102C00501D4
:1008E0000980A101850319012AB700150126B70067
:1008F000950175108100C0050C0901A1018504193D
:10090000012AA002150126A002950175108100C0E0
:1009100005010906A101050719E029E715002501D0
:100920009508750181029501750881010507190077
:1009300029FF150026FF0095067508810005081996
:10094000012905950575019102950175039101C075
:1009500011241FBECFEFDAE0DEBFCDBF04B603FE29
:1009600018C08091C3029091C402A091C502B091B9
:10097000C6028730904BA740B04B59F41092C30287
:100980001092C4021092C5021092C602E0E0F8E391
:10099000099511E0A0E0B1E0ECE9FBE402C00590AC
:1009A0000D92AC39B107D9F722E0ACE9B1E001C052
:1009B0001D92A33CB207E1F70E94EE170C94CC25E0
:1009C0000C940000FF93EF93E0919C01F0919D0146
:1009D000309709F00995EF91FF910895FC018591F9
:1009E000803011F0EFDFFBCF0895FF27E0E230E227
:1009F00047FF0CC0419597FF09C0EDE260957095E7
:100A000080959095611D711D811D911D27FF02C06C
:100A1000219530E350E2AA27660F771F881F991FA0
:100A2000AA1FA41710F0A41B63955A95A9F7AA3022
:100A300008F0A95FA05DAF93F3956115710581057D
:100A4000910541F7ED3211F4EF93F395F21718F495
:100A50003F93F395FBCF8F91B5DFFA95E1F70895BA
:100A6000E991F9918591803021F0853219F0AADF62
:100A7000F9CF089520E0E89455915532C1F35033F1
:100A800011F4689455915A3348F4505390F3220F5F
:100A9000022E220F220F200D250FF4CF0EF42195E8
:100AA00089919991533619F3533729F1533559F1F7
:100AB000BC0188279927E8945C3621F489919991A3
:100AC00068945591543639F446EF7EF077FF0DC0A7
:100AD0008FEF9FEF0AC055374AE039F0583540E1B3
:100AE00021F0523642E009F00895FF93EF937DDF45
:100AF000EF91FF91B7CFFF93EF93FC01819180308D
:100B0000B9F360DFFBCFFF93EF9368DFF1CFDF93A3
:100B1000CF93CDB7DEB72596A3DFCF91DF910895B0
:100B2000873A2DE5920721F0883A9D4541F00FC0A4
:100B3000FB018281882359F08BEE90E006C0FB0117
:100B40008281882321F088ED90E00E94590781E09E
:100B5000089581E008950C94900508950C94AD05D6
:100B60001F93CF93DF9300D000D01F92CDB7DEB795
:100B700049835A836B8330919F0189819A81311116
:100B800014C0662359F0222349F00E94AD0D182F9E
:100B9000682F89819A810E94560D03C00E94810DA1
:100BA000182F69817A81812F04C00E94AD0D69815F
:100BB0007A810F900F900F900F900F90DF91CF914F
:100BC0001F910C940715FC01262F408151816281F1
:100BD000738184810C94B00581E00895CF93DF93F5
:100BE000EC0160E00E94E305BE01DF91CF910C941F
:100BF000AE050C9481160C947D1608950E94000C8D
:100C00000E94FD052FEF84E39CE02150804090403E
:100C1000E1F700C000000C94DC1D0F931F93CF93ED
:100C2000DF938C0161E00E94E305EC01B8010E94B2
:100C3000AB05882309F45BC0B801CE010E94C71B35
:100C4000882309F454C0B801CE010E94FB17882301
:100C500009F44DC0B801CE010E94231B882309F47A
:100C600046C0F80182818823D9F1CF3D8CE5D807B1
:100C700079F140F4C115FCE5DF0791F0C130DC45A6
:100C800091F02EC0CC35EDE5DE0741F1CD35FDE527
:100C9000DF0709F1CB35DD4519F50E94441220C06C
:100CA0000E94FE0524C080915F02C82FC095C170CC
:100CB000C0FB80F980935F02CC2329F08DEF91E097
:100CC0000E94EE0414C08BEE91E00E94EE0410C06E
:100CD0000E94F2120CC00E943B1202C00E944712F6
:100CE000C801DF91CF911F910F910C94A905C0E02D
:100CF0008C2FDF91CF911F910F9108950E940E1DAF
:100D00000C94BD070E94C0070C94141DDF92EF9253
:100D1000FF920F931F93CF93DF93E82FF0E0E25FF2
:100D2000FD4FD490282F26952695269530E0F90181
:100D3000E255FD4F0491877010E0082E02C0159512
:100D400007950A94E2F701701127F901E256FD4F69
:100D5000E490F12C082E02C0F594E7940A94E2F78F
:100D600091E0E922FF24F901E257FD4FC491D0E060
:100D700002C0D595C7958A95E2F7C170DD270115A8
:100D8000110519F081EE0E944608E114F10419F0F2
:100D900086EE0E9446088D2D0E946309EF2819F007
:100DA00086EE0E94ED08012B19F081EE0E94ED08FD
:100DB000CD2B51F08CE2DF91CF911F910F91FF90DD
:100DC000EF90DF900C946309DF91CF911F910F9109
:100DD000FF90EF90DF900895EF92FF920F931F9393
:100DE000CF93DF938C01F62E8AE0E82EF8018491F0
:100DF000882309F457C0813009F042C0E8012196E8
:100E0000FE018491813031F42196FE0184910E948B
:100E1000630939C0823039F4E8012296FE018491D9
:100E20000E94460830C0833039F4E8012296FE0162
:100E300084910E94ED0827C0843029F5E8012296AC
:100E4000FE01249180E090E030E0205331092A3007
:100E5000310560F4E89EA001E99E500D1124C901FE
:100E6000840F951F2196FE012491EECF009759F033
:100E7000EFE9FFE03197F1F700C000000197F6CFEE
:100E80000E948606E8018E010F5F1F4F8F2D882379
:100E900009F4ACCFEFE9FFE03197F1F700C00000B3
:100EA0008150F5CFDF91CF911F910F91FF90EF907F
:100EB000089560E00C94EC068295982F937344E0BB
:100EC000949F900111248C7C86958695282B822FE7
:100ED0008575880F2A7A2695822B0895CF93DF9304
:100EE000D92F0E945C07C82F8D2F0E945C072C2FE2
:100EF00030E0322F2227A901482BCA01DF91CF9180
:100F00000895CF92DF92EF92FF920F931F93CF93AA
:100F1000DF936B017C01CB010E946E07EC01C701DE
:100F20000E946E07AC01CE01A0E0B0E0DC01992781
:100F3000882760E070E08C019D01042B152B262B87
:100F4000372BC901B801DF91CF911F910F91FF900D
:100F5000EF90DF90CF90089508950C94AC0781E056
:100F600008950C94AF070895CF93C82F0E94AD0742
:100F70008C2F0E94B107CF91089580E00C94B407A4
:100F80000E94231C0C94B407CF930E94231CC82FEB
:100F900080919E01C81741F1C0939E0180915F022C
:100FA00082FF1EC080FF04C085EC92E00E94EE0428
:100FB00080915F0280FF0CC01F92CF9380EC92E083
:100FC0009F938F930E9487050F900F900F900F9023
:100FD00080915F0280FF04C08EEB92E00E94EE04DD
:100FE0008C2FCF910C94B407CF910895CF93DF93BA
:100FF000CDB7DEB72B970FB6F894DEBF0FBECDBFCF
:101000004F83588769877A878B8761110E94731194
:101010009E012F5F3F4F86E0F90111928A95E9F713
:1010200085E0FE013796D90101900D928A95E1F78E
:1010300089819A814C815D81452B31F09F3F31F44C
:1010400091E08F3F19F403C091E001C090E090FF60
:1010500009C049815A816B817C818D819E810E946A
:10106000941005C0C9010E94EC058111F2CF2B96A6
:101070000FB6F894DEBF0FBECDBFDF91CF910895BC
:10108000FC01808191810E94EF0D0895CF93882308
:1010900009F4A1C0C82F8238C1F40E94231C81FD2D
:1010A0009AC069E380910201909103010E94E61CBD
:1010B0000E9495112FEF81EE94E0215080409040E6
:1010C000E1F700C0000069E319C0833801F50E9410
:1010D000231C80FD80C063E5809102019091030193
:1010E0000E94E61C0E9495112FEF81EE94E02150A2
:1010F00080409040E1F700C0000063E5809102016C
:10110000909103010E94E81CCF910C9495118438B2
:10111000C1F40E94231C82FD5EC067E4809102013D
:10112000909103010E94E61C0E9495112FEF81EE21
:1011300094E0215080409040E1F700C0000067E457
:10114000DDCF8CEF8C0F813AF8F48C2F0E94DA1AE5
:10115000811141C06C2F80910201909103010E9486
:10116000B01C882349F06C2F8091020190910301FB
:101170000E94E81C0E9495116C2F809102019091B1
:1011800003010E94E61CC0CF80E28C0F883048F437
:10119000C77081E001C0880FCA95EAF70E94561116
:1011A000B3CFEBE5EC0FE33040F4F0E0E15CFE4F51
:1011B000808190E0CF910C94781CC85AC73158F4C4
:1011C000EC2FF0E0EE0FFF1FEF5EFE4F808191816C
:1011D000CF910C948E1CCF910895882309F45BC0A5
:1011E000682F823879F40E94231C81FF54C069E380
:1011F00080910201909103010E94E61C0E949511CA
:1012000069E310C08338B1F40E94231C80FF43C0FF
:1012100063E580910201909103010E94E61C0E9407
:10122000951163E580910201909103010E94E81CF1
:101230000C949511843879F40E94231C82FF2BC0F2
:1012400067E480910201909103010E94E61C0E94D4
:10125000951167E4E7CF8CEF860F813A18F380E2AF
:10126000860F883048F4677081E001C0880F6A9566
:10127000EAF70E945C11DCCF8BE5860F833020F407
:1012800080E090E00C94781C685A673120F480E08C
:1012900090E00C948E1C08951F93CF93DF93182F2A
:1012A000EB010E944608209741F08FE99FE00197EB
:1012B000F1F700C000002197F6CF812FDF91CF9189
:1012C0001F910C94ED08893319F060E070E002C0C2
:1012D00060E570E00C944C09882321F00E945611BF
:1012E0000C9495110895882321F00E945C110C94B0
:1012F00095110895CF92DF92EF92FF920F931F9373
:10130000CF93DF937C01D62FC72FFC01128105817B
:1013100002950F700E944C118823B9F01123A9F097
:101320008C2F807F803421F080E28D0F883068F030
:101330008091810282FD09C082E00E94F5110E9425
:101340004C1191E0D82ED92601C0D12CCC2EC294BC
:101350008FE0C8228C2D90E08C30910508F0C4C13C
:10136000FC01EA5AFF4F0C9477258C2F807FCF70B9
:10137000882311F0C295C07F112399F0CC2309F482
:101380009FC180E28D0F883010F0D11104C08C2FE6
:101390000E94561103C08C2F0E9466110E94951165
:1013A0008FC18D2F0E94ED08CC2309F49DC180E2EE
:1013B0008D0F883038F1DD2329F18C2F0E946C11BC
:1013C00024C08C2F807FCF70803211F0C295C07FF7
:1013D000DD2319F0D130A1F13DC08091810282FF5F
:1013E00017C0112349F0CC2329F08C2F0E945611ED
:1013F0000E94951180E065C180E00E94ED08CC2339
:1014000009F472C18C2F0E945C110E9495116CC16D
:10141000112371F0002341F0013031F40E94761164
:101420008C2B0E947E1160C10E9476118C2B1DC0F6
:10143000002319F0013009F457C10E948B1125C017
:10144000112321F0063008F04FC10EC0053008F01E
:101450004BC11BC0112361F0002331F0F7018581DE
:1014600080FF2EC18F7085838C2F0E946C093CC138
:10147000002359F0D93309F034C1FFEF07EE13E030
:10148000F15000401040E1F72AC18C2F0E947309EF
:101490002BC18C2F86958695837019F0813061F071
:1014A00023C1112321F08D2F9C2F937002C080E067
:1014B00090E00E94781C20C1112321F08D2F9C2FD9
:1014C000937002C080E090E00E948E1C15C18C2FAA
:1014D000837009F047C011110BC12D2F229526955D
:1014E0002770220F220F6D2F6F70862F90E0A0E0E3
:1014F000B0E0022E04C0880F991FAA1FBB1F0A94D8
:10150000D2F7D4FF10C04FE050E060E070E004C0BC
:10151000440F551F661F771F2A95D2F740955095A7
:101520006095709503C040E050E0BA01C695C6953D
:10153000C3708A019B01082B192B2A2B3B2BC90155
:10154000B801C23049F058F4C13019F00E946C0C57
:10155000CFC00E945A0CCCC00E947E0CC9C00E9411
:10156000580CC6C0112319F08C2F817001C08695CC
:10157000882309F4BDC02D2F229526952770220FB0
:10158000220F6D2F6F70862F90E0A0E0B0E0022E4A
:1015900004C0880F991FAA1FBB1F0A94D2F7D4FF5B
:1015A00010C04FE050E060E070E004C0440F551FF1
:1015B000661F771F2A95D2F74095509560957095D4
:1015C00003C040E050E0BA01C695C695C3708A01D9
:1015D0009B01082B192B2A2B3B2BC901B801C230C8
:1015E00049F058F4C13019F00E94310D81C00E94B9
:1015F0001F0D7EC00E94430D7BC00E94920C78C0DC
:10160000CF70112339F08C2F0E94B80C8D2F0E94BF
:101610006C096EC08D2F0E9473098C2F0E94D90C0B
:1016200067C0D23F21F128F4D03F41F0D13FC1F053
:1016300043C0D33F19F1D43F79F03EC0112341F0AC
:10164000053008F051C08C2F8F710E94FE0C4CC0E9
:10165000063008F049C0F7CF8091810282FF18C0A0
:10166000112339F08C2F8F710E94B80C3DC01123CB
:10167000C9F38C2F8F710E94D90C36C0112329F029
:101680008C2F8F710E94A30C2FC00E949E0C2CC027
:10169000112349F0CF718C2F0E94B80C63E08C2F7E
:1016A0000E94DA1121C081E00E94F5110230E0F0C1
:1016B00082E00E94F51118C0112331F0002391F24D
:1016C0008D2F0E94460810C0002399F2D93349F4A7
:1016D0001FEF27EE33E0115020403040E1F700C00B
:1016E00000008D2F0E94ED0888EF8C0D843020F4CF
:1016F0000E94231C0E94B407DD20C9F00E944811FB
:1017000080FD15C0F70112820E9442110E94B80CA0
:10171000C7010E94B80B0E944211DF91CF911F9127
:101720000F91FF90EF90DF90CF900C94D90CDF9148
:10173000CF911F910F91FF90EF90DF90CF90089580
:101740000F931F93CF93DF93EC01688179818A8196
:101750000E94FA0D8C010E94550D0E94460CB801A2
:10176000CE010E947A09DF91CF911F910F910895C8
:10177000CF93DF93EC01988189812B813C81232BCE
:1017800031F08F3F31F481E09F3F19F403C081E0D5
:1017900001C080E080FD1DC0CE010E940D068111B8
:1017A00010C00E944C118823A1F08A81882389F0FF
:1017B0008091810282FD0DC082E0DF91CF910C9477
:1017C000F511CE010E94A00BCE01DF91CF910C94B8
:1017D000EE05DF91CF91089580E090E00E94781CA3
:1017E00080E090E00E948E1C0E9473110C94951171
:1017F00080910201909103010E94EA1C0C94EC0B71
:101800000E9463110C94F80B92959F70963079F0BA
:1018100010F4925001C09A50923068F4803F69F001
:1018200018F4883E40F409C0843F29F406C0883E7D
:1018300020F0813F11F080E0089581E00895FC01DF
:10184000808191810E94EF0D0E94040C0895CF9336
:10185000DF9300D000D01F92CDB7DEB70F900F906E
:101860000F900F900F90DF91CF910895CF93DF935A
:1018700000D000D000D0CDB7DEB726960FB6F894D2
:10188000DEBF0FBECDBFDF91CF91089508950895BB
:101890000C94470C0C94480C0E944A0C6093EF0186
:1018A0007093F0018093F1019093F2010C94EC0B92
:1018B0000C944C0C0F931F930091EF011091F001C9
:1018C0002091F1013091F201602B712B822B932B2F
:1018D0001F910F910C944C0C0F931F930091EF01EB
:1018E0001091F0012091F1013091F20160237123F8
:1018F000822393231F910F910C944C0C0F931F93F1
:101900000091EF011091F0012091F1013091F2016D
:1019100060277127822793271F910F910C944C0CFD
:101920000C94470C0E94900C6093EB017093EC01B7
:101930008093ED019093EE010C94EC0B60E070E06D
:10194000CB010C94920C0F931F9341E050E060E0A8
:1019500070E08A019B0104C0000F111F221F331F7A
:101960008A95D2F7C901B8011F910F910C94920C7E
:101970000F931F9341E050E060E070E004C0440F1B
:10198000551F661F771F8A95D2F78091EB019091C2
:10199000EC01A091ED01B091EE018A019B01082BB1
:1019A000192B2A2B3B2BC901B8011F910F910C94C5
:1019B000920C0F931F9341E050E060E070E004C090
:1019C000440F551F661F771F8A95D2F74095509593
:1019D000609570958091EB019091EC01A091ED01E3
:1019E000B091EE018A019B01082319232A233B238E
:1019F000C901B8011F910F910C94920C0F931F9382
:101A000041E050E060E070E004C0440F551F661FE5
:101A1000771F8A95D2F78091EB019091EC01A0910C
:101A2000ED01B091EE018A019B01082719272A27B1
:101A30003B27C901B8011F910F910C94920C0F9391
:101A40001F930091EB011091EC012091ED01309179
:101A5000EE01602B712B822B932B1F910F910C9415
:101A6000920C0F931F930091EB011091EC012091C8
:101A7000ED013091EE0160237123822393231F91A6
:101A80000F910C94920C0F931F930091EB01109106
:101A9000EC012091ED013091EE0160277127822742
:101AA00093271F910F910C94920C089523E1929F1C
:101AB000800D1124E82FE695E695E695877051E0B4
:101AC00001C0550F8A95EAF785E0E89FF0011124DF
:101AD000E056FE4F20E030E070E04081CB01022E66
:101AE00002C0969587950A94E2F7817081958427C4
:101AF0008523842781932F5F3F4F2530310569F778
:101B0000089523E1929F800D1124682F66956695B4
:101B10006695982F977085E0689FB001112440E08A
:101B200050E080E0FB01E40FF51FE056FE4F2081FE
:101B300030E0092E02C0369527950A94E2F721700D
:101B40003327042E01C0220F0A94EAF7822B4F5F3D
:101B50005F4F4530510531F70895BF92CF92DF9224
:101B6000EF92FF920F931F93CF93DF938C01C0905E
:101B7000EB01D090EC01E090ED01F090EE0180914E
:101B8000EF019091F001A091F101B091F201C82A0A
:101B9000D92AEA2AFB2ACFE1D0E0D701C6010C2ED0
:101BA00004C0B695A795979587950A94D2F780FDBE
:101BB00004C0219790F7B12C07C0BC2EB8018C2F20
:101BC0000E941A150197A9F38B2DDF91CF911F91D8
:101BD0000F91FF90EF90DF90CF90BF900895CF933B
:101BE000DF93EC010E94AD0DBE010E941A15DF913A
:101BF000CF9108951F93CF93DF93EB0190919F01B5
:101C0000992321F0CB010E94EF0D13C0882349F0E6
:101C1000CB010E94AD0D182F682FCE010E94560DEA
:101C200004C0CB010E94810D182FBE01812F0E949C
:101C30001A15DF91CF911F9108951F93CF93DF93D2
:101C4000C091F30116E08091F401C81799F0D0E03B
:101C50001C9FF0011D9FF00D1124EB50FE4F4081A1
:101C6000518162817381848195810E94360C219615
:101C7000C770E9CFDF91CF911F9108954091250260
:101C800050912602609127027091280280912902CA
:101C900090912A020C94360CEF92FF920F931F93AF
:101CA000CF93DF9380912A0282958F7009F065C0EF
:101CB00080912702882309F460C08091F301F0909D
:101CC000F401109125020091260260912802709182
:101CD000290291E01F3F09F090E0C0910001D091EE
:101CE0000101292F96E0E92E8F1509F446C06115F0
:101CF000710521F00F3F21F030E003C031E001C059
:101D0000322F90E030FD36C0E89EF001E99EF00DE4
:101D10001124DF01AB50BE4F11963C911197301347
:101D200029C03C91311326C012963C911297311173
:101D300021C013964D915C911497461B570B4C177D
:101D40005D07C0F480912A028F70806180932A021F
:101D5000E650FE4F80818F708061808385E292E043
:101D60000E94B80BDF91CF911F910F91FF90EF90E0
:101D70000C941D0E01968770B7CFDF91CF911F9104
:101D80000F91FF90EF9008959F92AF92BF92CF92E4
:101D9000DF92EF92FF920F931F93CF93DF93CDB714
:101DA000DEB761970FB6F894DEBF0FBECDBF8C01D2
:101DB00085E0F801DE011D9601900D928A95E1F70C
:101DC000D8011296EC9090912502E0912602209184
:101DD0002802309129022115310531F0EF3F31F40D
:101DE00081E09F3F19F403C081E001C080E0B82F7B
:101DF000B1709B2E80FD47C1D8014C9111965C912A
:101E000011971396AD90BC90149785E2C82E82E08E
:101E1000D82EF0902702B501621B730B20910001B0
:101E200030910101FF2009F4D9C080912A02621784
:101E3000730708F095C0282F207F09F052C05E1369
:101E400013C0491311C0FE2CE1100EC08F708061C9
:101E500080932A020E943E0EC6010E94B80B809118
:101E60002A02F80185834DC1AB2831F05F3F31F480
:101E700081E04F3F19F403C081E001C080E080FDA4
:101E800003C081E08E2502C080E090E0F82FF17061
:101E9000FF2E80FF1CC08091F3012091F40136E0F9
:101EA000821709F40BC190E0389FF001399FF00DC3
:101EB0001124EB50FE4F6181561306C0608146131A
:101EC00003C06281E61203C001968770E9CFFE2C41
:101ED000EE2009F416C180912A02816080932A02C3
:101EE00054C05E1306C0491304C0E11002C0F801DB
:101EF00099C0C8010E941F0C882361F1EE2051F1A6
:101F000020912A02822F82958F7090E0029774F0C0
:101F1000809125029091260298878F831986BB862F
:101F2000AA862C87CE0107960E94B80B86E0F8019E
:101F3000A5E2B2E001900D928A95E1F70E944C0E65
:101F40000E943E0E0AC05E1711F1C8010E941F0CCC
:101F500081112CC0C8010E94B80BFF24F394D1C09A
:101F6000282F207F81F77A2DB98AA88A6E2D89893A
:101F70000E94270C85E292E00E94B80B86E0D60111
:101F80001D928A95E9F70E943E0EF12CBAC04913C2
:101F9000DCCFE110DACFF8018583C8010E94B80BCD
:101FA00086E0D6011D928A95E9F7ABC0EE2091F24A
:101FB00020912A02822F82958F7090E002970CF474
:101FC000B5CF80912502909126029A8389831B8246
:101FD000BD82AC822E83CE010196A6CF6217730715
:101FE00008F044C0FE2CEE2009F4B4CF5E1330C0DC
:101FF00049132EC020912A0220FD21C0822F8295F4
:102000008F70482F50E041155105C9F0F801258324
:102010004F30510541F08F5F982F9295907F822F1E
:102020008F70892B8583C8010E94B80B86E0F80168
:10203000A5E2B2E001900D928A95E1F73CC086E0FE
:10204000F801A5E2B2E001900D928A95E1F759C03E
:10205000C8010E941F0C811169CF80912A02816002
:1020600080932A02C8010E94B80B4BC07A2DB98A0E
:10207000A88A6E2D89890E94270C86E0D6011D92C0
:102080008A95E9F718C0EE2009F464CFC8010E94D0
:102090001F0CF82E882309F45DCF86E0F801A5E235
:1020A000B2E001900D928A95E1F785E292E00E94FC
:1020B00040080E944C0E0E943E0E23C04D875E8752
:1020C0008D859E850E94EF0D292F22952F7022303D
:1020D00028F49F7039F0811105C00BC0243028F41A
:1020E0009F7049F4805E883020F0C8010E94B80BD0
:1020F0009F2CF92C06C0D80115969C91907F91F7E2
:10210000F8CF8F2D61960FB6F894DEBF0FBECDBF0E
:10211000DF91CF911F910F91FF90EF90DF90CF90C3
:10212000BF90AF909F9008951F93CF93DF93CDB74B
:10213000DEB72C970FB6F894DEBF0FBECDBF4F832E
:10214000588769877A878B879C87CE0107960E947C
:10215000C40E8823D1F09F8188852A853B85232B57
:1021600031F08F3F31F481E09F3F19F403C081E0EB
:1021700001C080E080FD47C04F81588569857A8520
:102180008B859C850E94360C3EC086E0FE0137960A
:10219000DE01119601900D928A95E1F7FF81E885A5
:1021A0006A857B856115710531F0EF3F31F481E07F
:1021B000FF3F19F403C081E001C080E080FD23C02F
:1021C0002091F40130E0C901019687709927409170
:1021D000F30150E084179507F1F1F983EA837D83D9
:1021E0006C8396E0929FD001939FB00D1124AB5069
:1021F000BE4FFE01319601900D929A95E1F78093C2
:10220000F4010E941D0E16E08091F3019091F401FB
:10221000891771F1189FC00111248B509E4F0E94A5
:10222000C40E882329F1E091F3011E9FF0011124CF
:10223000EB50FE4F40815181628173818481958191
:102240000E94360C8091F30190E0019687709927E7
:102250008093F301D9CF0E94000C1092F4011092E8
:10226000F301E5E2F2E086E0DF011D928A95E9F7ED
:102270002C960FB6F894DEBF0FBECDBFDF91CF9185
:102280001F910895809133028595859585950895D0
:10229000809133028770089590913302977081E0A6
:1022A00009F480E0089580913E02089590913E02E5
:1022B000892B80933E020895809590913E02892358
:1022C00080933E02089510923E02089590913D023F
:1022D000892B80933D020895809590913D0289233A
:1022E00080933D02089510923D020895809134023A
:1022F000089508950C9479110C947A1190918102AB
:1023000092FD08C090913402981721F08093340216
:102310000C947C11089580913402882329F0109246
:10232000340280E00C947C110895CF93DF93E09108
:102330000201F091030180913E028083E09102014D
:10234000F0910301908180913D02892B80838091DF
:102350003402882381F0E0910201F0910301908121
:10236000892B808380910201909103010E94A41C1B
:1023700081110E948B11C0910201D091030148E0AC
:1023800050E06BE272E0CE010E947D25892B69F05E
:1023900088E0FE01ABE2B2E001900D928A95E1F790
:1023A000CE01DF91CF910C942F1CDF91CF91089536
:1023B0000C9479119091810292FD10C098E0899F50
:1023C00090011124262B209333020E94B80C809197
:1023D00033028595859585950C94D8110C94B80C8D
:1023E0001092330280E00C94D81120913302809532
:1023F000822380933302982F977099F430E0482F0E
:10240000082E000C550B2417350759F090918102C6
:1024100092FD07C08595859585950E94D90C0C94F1
:10242000F0110895CF939091810292FB222720F919
:102430002817F9F0C82F892FC0FB82F980938102F9
:1024400080918002909181020E946E1282E00E942F
:10245000F51180915F0280FF0CC01F92CF9380ED39
:1024600092E09F938F930E9487050F900F900F909B
:102470000F90CF9108958091810282FB882780F987
:1024800091E089270C94121281E00C94121280E0E2
:102490000C94121280E090E00E94922521E0893E87
:1024A0009E4F09F020E0822F089582E090E00C9486
:1024B0008A2583E090E00C948A25CF9384E090E015
:1024C0000E948A25C82F82E290E00E948A252C2F44
:1024D00030E0A901582BCA01CF910895CF93C92F9D
:1024E000682F84E090E00E9498256C2F82E290E0B3
:1024F000CF910C949825AB01BC018FE090E00C9437
:10250000AA25AB01BC0183E190E00C94AA2560E010
:1025100070E0CB010C94811260E070E0CB010E946E
:102520007B120C94871269EE7EEF80E090E00E94AF
:10253000B62560E082E090E00E94982560E083E0AC
:1025400090E00E9498251092EF011092F0011092F5
:10255000F1011092F20160E084E090E00E94982581
:1025600060E082E290E00E94982560E085E090E0E3
:102570000E94982560E086E090E00E9498256FEF29
:1025800087E090E00E94982540E050E0BA0188E0A2
:1025900090E00E94AA2560E08DE090E00E949825DE
:1025A00040E050E0BA0188E190E00E94AA2560E096
:1025B00087E190E00E94982540E050E0BA018CE16C
:1025C00090E00E94AA2560E070E080E290E00E9426
:1025D000B62540E050E0BA0188E190E00E94AA25CB
:1025E0000C948C120C949312682F8EE090E00C9453
:1025F00098250E949B1D60935B0270935C02809300
:102600005D0290935E02609357027093580280932C
:10261000590290935A02089585B7806885BF85B79F
:10262000806885BF089581E008950C941313089580
:102630000C9417130C9417130C941A130C9417136F
:102640000C941E130C9417130E940C1385EB9FE13E
:102650000E94191C0E9422130C9420130E9418132C
:102660000C9417130E94F7150C94B3070E94861D53
:102670000E9445170E9432130C941C132F923F9214
:102680004F925F926F927F928F929F92AF92BF9282
:10269000CF92DF92EF92FF920F931F93CF93DF932E
:1026A000CDB7DEB72D970FB6F894DEBF0FBECDBF06
:1026B0000E945A17282E81110E94F9128FE392E08E
:1026C0009D878C8700E010E0302E802F0E941B1623
:1026D0002B013C01EC85FD8581919191A191B191F6
:1026E000FD87EC875301420188269926AA26BB263E
:1026F00081149104A104B104B1F40F5F1F4F06309F
:10270000110511F78FEF89838A831B820E948F1D29
:102710008160782F9D838C8349815A816B818D8163
:102720000E94F60751C080915F0281FD0E9427162A
:102730001B86C12CD12C7601C394D501C4018C21F8
:102740009D21AE21BF21892B8A2B8B2B91F10E94D9
:1027500015138823D1F0FB85FE833F824C205D203A
:102760006E207F2081E045284628472809F480E034
:1027700088870E948F1D8160782F9A8789874E8174
:102780005F8168858A850E94F607000F111F000F80
:10279000111FF801E15CFD4F80819181A281B3811D
:1027A000C826D926EA26FB26C082D182E282F3829D
:1027B0000BC08B858F5F8B87CC0CDD1CEE1CFF1C48
:1027C000833109F0BACF99CF81E0211001C080E0B8
:1027D0002D960FB6F894DEBF0FBECDBFDF91CF911F
:1027E0001F910F91FF90EF90DF90CF90BF90AF902F
:1027F0009F908F907F906F905F904F903F902F9021
:1028000008950E943E130C94C407CF93DF930E9457
:102810001F15EC01811522E59207E8F5811531E5D8
:10282000930708F0B6C0883E910528F5803E9105D3
:1028300008F0E9C0883A910570F4853A910508F0EE
:102840007AC08130910509F473C008F4D9C00497A7
:1028500008F0D9C0D5C08F3B910508F0D1C0C85A47
:10286000D0E0CC0FDD1FCE5BDE4F0990D881C02DAC
:10287000CE019464C9C0811540E5940708F069C091
:10288000811550E4950708F060C09A9581159F4125
:1028900008F4B9C0B5C0811536E5930728F5811550
:1028A00045E5940708F092C0811554E5950708F0B6
:1028B00087C0AC0143705527282F26952695C11552
:1028C000D34508F06CC081E090E002C0880F991FEA
:1028D0004A95E2F740E2249F90011124EC01C22BBB
:1028E000D32BCE019C6890C081152AE5920780F415
:1028F000811539E5930708F072C0811548E5940702
:1029000008F47EC0D82FCC27CE01806F906A7CC09F
:1029100090568115904208F073C08D2F8F710E94E0
:10292000B315DD27D0628F71AE01582BCA016CC080
:1029300081E090E069C0C55AD0E0C059DE4F88817F
:10294000C82FD0E0CE0190645FC0DF70CE01906AE6
:102950005BC074E0969587957A95E1F7282F2370F0
:102960003C2F337081E090E002C0880F991F3A95A8
:10297000E2F79C68AC01522B9A019C2F9F709695B0
:10298000969550E2959FE0011124C9018C2B9D2B57
:102990003BC0D82FCC27CE01816F906A35C081E033
:1029A00090E002C0880F991F4A95E2F750E2259FF8
:1029B00090011124EC01C22BD32BCE019A6824C0C4
:1029C000D82FCC27CE01846F906A1EC00E94B31509
:1029D0008F7190E0D82FCC27CE01906215C08F70F8
:1029E0000E94B31594E0D695C7959A95E1F7CF70FC
:1029F000D0E0DC2FCC27D0699E01282BC90104C070
:102A000080E090E001C0CE01DF91CF91089522E7F0
:102A1000829FC0011124FC0123E1729FE00DF11D92
:102A20001124E60FF11DEE0FFF1FE95FFE4F8591A8
:102A3000949108950E9407150E9405140895823804
:102A4000910569F1B0F48133910509F46DC048F442
:102A50008932910509F463C08A32910509F469C08D
:102A600008958533910509F455C089339105B9F06E
:102A70000895833E910569F138F4803E9105B1F0E7
:102A8000823E910509F10895863E9105A9F1873EA0
:102A90009105B9F1843E910509F064C023C02091ED
:102AA000800220FD4FC021FD4DC00895809180021D
:102AB00080FD44C08091810280FF44C080918002EB
:102AC00084FD42C083EE4DC08091800282FF38C0F9
:102AD000F5CF8091800282FD33C08091810280FD1C
:102AE00031C0ECCF8091810281FF32C080918002A1
:102AF00084FD2AC087EE35C08091800283FF26C006
:102B0000F5CF8091800283FD21C08091810281FDFB
:102B10001FC0ECCF8091800285FD1CC01DC080913C
:102B2000800285FD19C016C08091800286FD16C006
:102B300017C08091800286FD13C010C089E311C0C8
:102B400082EE0FC080EE0DC080E00BC086EE09C0A3
:102B500084EE07C089E205C085E303C08AE201C0B4
:102B600081E390E008959091800292FF0DC0282F9C
:102B70002871283019F4877F846006C0282F2471BB
:102B8000243011F48B7F886093FF0DC0282F2871AB
:102B9000283119F4877E846106C0282F24712431DE
:102BA00011F48B7E88612091810220FF0DC0382FA7
:102BB0003871383019F4877F816006C0382F317141
:102BC000313011F48E7F886021FF0DC0282F2871CD
:102BD000283119F4877E816106C0282F21712131A7
:102BE00011F48E7E886194FD877E089508950E9479
:102BF0004A12811102C00E94F2120E945512809363
:102C00005F020E945D1290938102809380020E9475
:102C1000F6150E945912682F70E080E090E00E9443
:102C2000580C6091EB017091EC018091ED01909155
:102C3000EE010C94900C24E0829FC0011124FC0151
:102C4000E656FD4F60817181828193810895CF9214
:102C5000DF92EF92FF920F931F93CF93DF9386EF54
:102C600092E00E94EE048AE9E82E82E0F82EC0E0AD
:102C7000D0E091EFC92E92E0D92E07EE12E0DF935B
:102C8000CF93DF92CF920E9487058EEE92E00E9452
:102C9000EE04F70161917191819191917F010E9400
:102CA00081079F938F937F936F931F930F930E943E
:102CB000870585EE92E00E94EE0421968DB79EB7BF
:102CC0000A960FB6F8949EBF0FBE8DBFC630D105D1
:102CD000B1F6DF91CF911F910F91FF90EF90DF90B0
:102CE000CF90089580EA8A95F1F7089500C008957D
:102CF0000C94721608950C947A160C947B160C940E
:102D00007A160C947F16F894E82FE295EF70F0E0B5
:102D100031A1282F2F7081E090E001C0880F2A9503
:102D2000EAF7982F9095932391A392A1892B82A3E0
:102D3000789408950F931F93CF93DF93C6E8D1E063
:102D400089918F3F11F00E94831681E0CC38D8071B
:102D5000B9F7C3E7D1E006E811E089918F3F11F0A0
:102D60000E9483160C171D07C1F7DF91CF911F91A9
:102D70000F9108954F925F926F927F928F929F92E0
:102D8000AF92BF92DF92EF92FF920F931F93CF9378
:102D9000DF938C01C62FD0E0CE018A579E4F7C0175
:102DA000FC0190819F3F09F460C0D62EF894E92F72
:102DB000E295EF70F0E081A19F7021E030E001C06A
:102DC000220F9A95EAF7822B81A382A120952823CE
:102DD00022A378940E947616E3E7F1E026E831E03A
:102DE000412C512C32014394812C912C540181911E
:102DF0008F3F99F0A82FA295AF70B0E090964C91BC
:102E000050E08F70BA0102C0759567958A95E2F718
:102E100060FD03C0D301C20103C080E090E0DC018B
:102E2000882A992AAA2ABB2A440C551C661C771C9E
:102E30002E173F07E1F6F70180818F3F11F00E94C6
:102E4000831661E081149104A104B10409F460E0E7
:102E50008D2D0E947816CC0FDD1FCC0FDD1FC00F0B
:102E6000D11F88829982AA82BB82DF91CF911F9164
:102E70000F91FF90EF90DF90BF90AF909F908F9059
:102E80007F906F905F904F9008950E949A1688E10E
:102E9000EAE9F2E0DF01982F1D929A95E9F7E2E85E
:102EA000F2E0DF011D928A95E9F786E00E94A517FE
:102EB0000C94F905FF920F931F93CF93DF93CDB737
:102EC000DEB768970FB6F894DEBF0FBECDBF8E0198
:102ED0000F5F1F4F88E1F80111928A95E9F7F12CF5
:102EE0006F2DC8010E94BA16F394F6E0FF12F8CFD6
:102EF00048E150E0B80182E892E00E947D25FF247D
:102F0000F394009709F4F12C892B41F088E1F80142
:102F1000A2E8B2E001900D928A95E1F72F2D46E0EC
:102F20006AE972E082E892E00E94A6170E94FB051F
:102F30008F2D68960FB6F894DEBF0FBECDBFDF9120
:102F4000CF911F910F91FF9008950895FF920F93D5
:102F50001F93CF93DF93F82ED92F8B01C42F2223F9
:102F600049F081E0809362020E948F1D909361027C
:102F700080936002809162028823F1F08091600268
:102F8000909161020E94A71D0597B0F0EF2DFD2FD3
:102F9000D80180E090E04C2F50E08417950754F45E
:102FA00001911191219131910D931D932D933D9399
:102FB0000196F3CF10926202DF91CF911F910F9192
:102FC000FF9008950E9431200E9436130C943D20FA
:102FD0000E9441200E9401140C945F200E942D1D2C
:102FE0000E9418200E9424130E94E2170E94E817F2
:102FF0000E942E13FBCFCF93DF93EC01FB01828164
:10300000882309F43CC1C430FDE5DF0760F4CB3F01
:103010009CE5D90788F49E0122503C4524313105B6
:1030200008F02EC109C0C236EDE5DE0729F0C63A28
:10303000FDE5DF0709F024C10E945D129093810233
:1030400080938002C1318CE5D80709F4C6C008F02E
:1030500042C0C930ECE5DE0709F49BC000F5C5307D
:103060008CE5D80709F485C078F4C330ECE5DE07B9
:1030700009F478C008F07AC0C230DC4509F0F5C028
:10308000809180028160EFC0C7309CE5D90709F4C8
:1030900078C008F07AC0809180028061E4C0CD30B1
:1030A000FCE5DF0709F487C058F4CB309CE5D9076D
:1030B00009F479C008F07BC08091800288606FC0FD
:1030C000CF30FCE5DF0709F480C008F082C08091B2
:1030D0008002877FC8C0CE3F9CE5D90709F471C044
:1030E00000F5C531FCE5DF0709F485C068F4C3319C
:1030F0009CE5D90709F475C008F095C00E94000C42
:10310000809180028F77AFC0CC3FFCE5DF07A9F14B
:1031100008F054C0CB3FDC4509F0A7C08091810284
:1031200040C0C230EDE5DE0709F489C058F4C1158E
:103130008DE5D80709F45AC008F069C08091810272
:1031400082602FC0C236EDE5DE0709F47CC0C63AC6
:10315000FDE5DF0709F481C0C330DD4509F085C016
:1031600080E06EC08091800282607DC0809180028C
:1031700016C080918002886076C080918102826052
:103180004FC08091800280626EC080918002806416
:103190006AC00E94000C80918002806864C08460D4
:1031A00062C081603DC0809180028E7F5CC0809152
:1031B00080028D7F58C08091800216C0809181026C
:1031C00018C0809181028D7F2BC0809180028F7EFC
:1031D0004AC0809180028F7D46C0809180028F7BA3
:1031E00042C080918002877F8B7F3DC080918102A9
:1031F0008D7F8E7F15C08091800282FB222720F96F
:1032000091E0922790FB82F990FB83F92CC080918A
:103210008102982F909591708E7F892B90FB81F978
:103220008093810222C00E94000C8091800287FB63
:10323000222720F991E0922790FB87F914C081E0C2
:103240000E94F41212C08091800284FB222720F990
:1032500091E0922790FB84F906C080918002982F1C
:10326000909590FB80F980938002809180029091EC
:1032700081020E946E120E94000C80E001C081E079
:10328000DF91CF910895CF93C82F1F928F9383E240
:1032900093E09F938F930E94870581E090E0A0E0E8
:1032A000B0E0BC01CD0104C0660F771F881F991FD5
:1032B000CA95D2F70E94580C0F900F900F900F9064
:1032C000CF910C94000CEF92FF920F931F93CF932A
:1032D000DF938B3109F4EDC008F08EC08B3009F418
:1032E000B1C008F078C0863009F4AFC020F4853052
:1032F00009F4BDC04EC1873009F4C0C0883009F060
:1033000048C10E9459121F928F9383E397E09F93C5
:103310008F930E9487050E94551283FB992790F98D
:103320001F929F9382FB992790F91F929F9381FB95
:10333000992790F91F929F93982F91701F929F93B6
:103340001F928F938AEE96E09F938F930E9487053A
:103350000E945D1287FB222720F91F922F9386FB84
:10336000222720F91F922F9385FB222720F91F92F5
:103370002F9384FB222720F91F922F9383FB222770
:1033800020F91F922F9382FB222720F91F922F935F
:1033900091FB222720F91F922F93292F21701F9232
:1033A0002F9381FB222720F91F922F93282F217022
:1033B0001F922F939F938F9385E096E09F938F9317
:1033C0000E9487058DB79EB788960FB6F8949EBF6A
:1033D0000FBE8DBF35C0803109F495C020F48E300A
:1033E00009F47BC0D6C0863109F4A8C0893109F040
:1033F000D0C083E993E084C08A32E1F060F4873280
:1034000009F4C3C028F48E3108F4C3C08D51BEC086
:10341000893269F1BEC0833448F48A3308F0B3C0FE
:10342000853309F4B2C0883369F0B3C0833409F43A
:10343000ACC0AFC08EED97E00E94EE040E94F21285
:10344000C1E0ACC082E694E05BC080915F02817F06
:103450008E7F80935F0287E494E00E94EE048AED01
:1034600097E00E94EE0481E080936302E9CF8EEB47
:1034700097E00E94EE040E94FE05E2CF80915F0279
:10348000C82FC095C170C0FB80F980935F02CC2328
:1034900029F082EB97E00E94EE0480C085EA97E075
:1034A0000E94EE0480915F02897F877F80935F0294
:1034B000C7CF90915F0291FBCC27C0F981E0C8276C
:1034C000892FC0FB81F980935F02CC2319F088E932
:1034D00097E029C08AE897E013C090915F0292FBC1
:1034E000CC27C0F981E0C827892FC0FB82F98093DF
:1034F0005F02CC2319F08BE797E015C08BE697E0CD
:103500000E94EE049DCF90915F0293FBCC27C0F9FF
:1035100081E0C827892FC0FB83F980935F02CC2309
:1035200051F08FE597E00E94EE0480915F02816088
:1035300080935F0233C082E597E0E2CF0E949B1D3B
:10354000162F072FF82EE92ED0917F02C09110017F
:103550000E94231CEF92FF920F931F931F92DF9301
:103560001F92CF931F928F9388E293E09F938F9344
:103570000E9487058DB79EB70C960FB6F8949EBF34
:103580000FBE8DBF5DCF895301C080E00E944319FB
:1035900057CF80E597E00E94EE04C0E08C2FDF91CA
:1035A000CF911F910F91FF90EF90089580E00895C3
:1035B0000C94D61ACF93C82F80916302882319F0F8
:1035C000813031F038C00E9453118232B1F504C00D
:1035D0000E945311823261F48C2F0E94D81A8111FB
:1035E00004C08C2F0E94631924C081E090E021C0A8
:1035F0008C2F0E94D61A81111BC0C43189F018F497
:10360000CB3029F010C0C93259F0C83361F487E4D7
:1036100094E00E94EE048FE193E00E94EE0408C063
:10362000109263020CC08DE193E00E94EE0407C08B
:1036300081E0817006C01092630280E002C080E0E9
:10364000F8CFCF910895CF93DF9386319C4541F514
:10365000EB010E945311982F8A8120910201309131
:103660000301882379F09A7A81E009F480E080935D
:103670006402911102C069E201C065E3C9010E94C0
:10368000E61C0AC080916402811102C069E201C097
:1036900065E3C9010E94E81C0E94951180E001C009
:1036A00081E0DF91CF9108950F931F93CF93DF9324
:1036B000C42FD22FFC0182818823C9F04093670276
:1036C0000E948F1D909366028093650280E28C0FAA
:1036D000883008F057C0C77081E001C0880FCA95D4
:1036E000EAF7DF91CF911F910F910C946C098091B3
:1036F0006702481330C080916502909166020E9473
:10370000A71D883C910538F510E21D0FCD17B9F0C3
:1037100080E28C0F883040F4C77081E001C0880FD0
:10372000CA95EAF70E947309183028F581E09D2FA9
:10373000977001C0880F9A95EAF70E946C09802F54
:103740000E9463091830F0F4D77081E001C0880F3F
:10375000DA95EAF70AC080E28C0F883098F4C770D7
:1037600081E001C0880FCA95EAF7DF91CF911F91E0
:103770000F910C947309802FDF91CF911F910F91BE
:103780000C946309DF91CF911F910F9108950F93CE
:103790009C01CB01243F4CE5340731F188F4293DED
:1037A000FCE53F07D9F02A3D4CE5340779F1283D87
:1037B0003C45A9F506E221EE41EE68ED7CE52BC023
:1037C000263FFCE53F07E1F0A8F0273F3C4539F5EF
:1037D00007E225EE46EE67EF7CE51DC007E225EE29
:1037E00045EE69ED7CE517C006E221EE40EE64EFA0
:1037F0007CE511C007E225EE44EE65EF7CE50BC0E9
:1038000006E221EE42EE66EF7CE505C008E221E02B
:1038100045EE6AED7CE50E94541B80E008C0FC0187
:103820008281882319F01092670201C081E00F9114
:10383000089590939D0180939C01089590936D024B
:1038400080936C020895E0916C02F0916D023097C4
:1038500021F00190F081E02D099480E00895EF922D
:10386000FF920F931F93CF93DF93E0916C02F0913F
:103870006D023097B1F18C010280F381E02D099542
:1038800080915F0282FF2DC080FF04C087EF97E028
:103890000E94EE04E80118E081EFE82E87E0F82EA0
:1038A00080915F0280FF0BC088811F928F93FF92EF
:1038B000EF920E9487050F900F900F900F9011507C
:1038C00021961111EDCF80915F0280FF0AC08FEE2B
:1038D00097E0DF91CF911F910F91FF90EF900C94A3
:1038E000EE04DF91CF911F910F91FF90EF9008951B
:1038F00020916A0230916B022817390771F090937A
:103900006B0280936A02E0916C02F0916D02309735
:1039100021F00680F781E02D099408952091680236
:10392000309169022817390771F0909369028093EA
:103930006802E0916C02F0916D02309721F00084F2
:10394000F185E02D09940895FC01329697E080E01E
:10395000915029F021912223D9F38F5FF9CF089557
:10396000662349F0FC01329608962191621729F0EE
:10397000E817F907D1F780E0089581E008959C01E8
:10398000FC0132969FEF80E04191461789F09F3FFE
:1039900019F4411101C0982F8F5F8630A9F79F3F1E
:1039A00039F0F901E90FF11D97FDFA956283089549
:1039B00008959C012A5F3F4FFC014281461301C0DC
:1039C0001282019682179307B9F708950C94BF1CD1
:1039D0000C94D91C029626E0FC0111922A95E9F775
:1039E000089508950C94F11C83E080936E020C946A
:1039F000F21C811102C081E001C082E080936E025E
:103A00000C94F21C0C94F91C81E080936E020C94CF
:103A1000F21C0C94041D08950C940B1D0C940C1DA9
:103A20000C940B1D0C940B1D0C940B1DCF930E943A
:103A3000121D0E945A170E94101DC0E08C2F0E9478
:103A40001B16672B682B692B29F4CF5FC630B1F7A3
:103A500080E001C081E0CF91089508951F920F92F8
:103A60000FB60F9211248F939F93AF93BF938091C2
:103A70006F02811113C08091B2029091B302A091A4
:103A8000B402B091B5024196A11DB11D8093B2025E
:103A90009093B302A093B402B093B502BF91AF91DB
:103AA0009F918F910F900FBE0F901F90189580914E
:103AB000BA02843031F10E947E0610926F0220E437
:103AC00088E190E00FB6F894A895809360000FBE4F
:103AD0002093600083B7817F846083BF83B7816058
:103AE00083BF7894889583B78E7F83BF0FB6F89491
:103AF000A8958091600088618093600010926000BA
:103B00000FBE08950E94000C0C94820682E084BDD2
:103B100093E095BD9AEF97BD80936E0008952FB7FF
:103B2000F8948091B2029091B302A091B402B09146
:103B3000B5022FBF08952FB7F8946091B20270912B
:103B4000B3028091B4029091B5022FBF08959C01F9
:103B50004FB7F8948091B2029091B302A091B40251
:103B6000B091B5024FBF821B930B089578941F92BA
:103B70000F920FB60F9211248F939F93AF93BF9321
:103B80008091B2029091B302A091B402B091B502BB
:103B90000196A11DB11D8093B2029093B302A09330
:103BA000B402B093B502BF91AF919F918F910F90E6
:103BB0000FBE0F901F90189581E08093E00080E287
:103BC0008093D8001092C9008FE19EE40197F1F72D
:103BD00000C0000087E090EBDC018093C30290936B
:103BE000C402A093C502B093C6029CE088E10FB660
:103BF000F894A895809360000FBE90936000FFCF6B
:103C000080917E0208950895CF93DF9321E0209361
:103C1000E9002FEF3091E800215035FD06C035ED69
:103C20003A95F1F700002111F5CF2091E80025FF2A
:103C300014C0EC0140E050E068E070E00E94CE204B
:103C40008091E8008E778093E80088E0FE01A6E787
:103C5000B2E001900D928A95E1F7DF91CF9108953E
:103C60008093720270937402609373028091BA021F
:103C7000843001F582E08093E9008FEF9091E800B5
:103C8000815095FD06C095ED9A95F1F700008111E0
:103C9000F5CF8091E80085FF0DC040E050E063E083
:103CA00070E082E792E00E94CE208091E8008E775B
:103CB0008093E8000895BC0184E00C94301EBC01A0
:103CC00083E00C94301E08958DE198E00E94EE048C
:103CD0008091B902811109C00E945F220E94BC221A
:103CE0008091E20084608093E200089589E198E089
:103CF0000E94EE041092B902089585E198E00E94B6
:103D0000EE040C94091D81E198E00E94EE0460919C
:103D1000B60281E0611101C080E00C94F41C8DE0DA
:103D200098E00E94EE049091BA0281E0943009F08C
:103D300080E06091B6020C94F91C209171022F5F13
:103D4000822F62E30E946B25992319F02093710260
:103D500008951092710280917502882371F180910B
:103D6000BA02843041F58091E9008F702091EC0017
:103D7000922F917020FD90E8892B93E09093E900B9
:103D80009091EB0090FF14C09091EE0097FF10C04F
:103D90009091E80095FF03C01092F100F9CF909147
:103DA000E80090FF05C09091E8009E779093E800AE
:103DB0008F708093E90010927502089542E061ECE3
:103DC00081E00E94D82142E261EC82E00E94D82189
:103DD00042E261EC83E00E94D8219091BA0281E036
:103DE000943009F080E06091B6020C94021D80913D
:103DF000BC02833009F461C030F4813071F082304C
:103E000009F49AC008958A3009F486C08B3009F409
:103E10006CC0893009F0A8C020C08091BB02813AF3
:103E200009F0A2C08091E800877F8093E80080912C
:103E3000BF029091C002892B21F468E086E792E0EE
:103E400003C060E080E090E070E00E941921809162
:103E5000E8008B778093E80008958091BB0281325F
:103E600009F082C08091BF029091C002029708F0D1
:103E70007BC08091E800877F8093E8008091E80014
:103E800082FD05C08091BA028111F8CF6DC02091EA
:103E9000F3008091F20090E0922B029731F4809130
:103EA000F100813011F0863021F48091F10080938F
:103EB0007E028091E8008B7753C08091BB02813AEB
:103EC00009F052C08091BF029091C002892B09F085
:103ED0004BC08091E800877F8093E8008091E800E4
:103EE00080FFFCCF8091100136C08091BB028132EF
:103EF000D9F58091BF029091C002892BA9F58091DC
:103F0000E800877F8093E8000E940D228091BD0227
:103F1000809310010C94000C8091BB02813221F53A
:103F20008091E800877F8093E8000E940D228091B5
:103F3000BE0280937F0208958091BB02813AA1F472
:103F40008091E800877F8093E8008091E80080FFFF
:103F5000FCCF80917F028093F1008091E8008E7702
:103F60008093E8000C940D2208959FB7F894109266
:103F700075029FBF9091BA02943009F057C090919A
:103F8000E9009F703091EC00232F217030FD20E874
:103F9000922B23E02093E9002091EB0020FF43C007
:103FA0002091EE0027FF3FC020917002222321F0D4
:103FB0002091E80025FF37C01092700226E0309172
:103FC000E80035FD15C03091BA02343061F530910A
:103FD000EB0035FD28C0215021F481E08093700270
:103FE00022C0EFE9FFE03197F1F700C00000E7CF12
:103FF0008093F1008091E80085FD0AC08091E8007F
:1040000080FFFCCF8091E8008E778093E80006C0A7
:104010008FB7F89421E0209375028FBF9F70909323
:10402000E90080E008959F709093E9008FEF089574
:1040300084B7877F84BF0FB6F894A89580916000FD
:10404000886180936000109260000FBE90E080E86D
:104050000FB6F89480936100909361000FBE0C94AA
:10406000041D0E945F220E94BC22E2EEF0E08081EB
:104070008460808378940C94502584E091E00C94C3
:104080001E1C8091BA028530C9F489E098E00E9434
:10409000EE048091BA02853079F40E94571D809118
:1040A000B8028823B1F30E94161D882391F30E9461
:1040B000B8200E94000CEDCF0C94821D0895089545
:1040C0000C946220292F332723303105C9F060F486
:1040D0002130310581F02230310509F041C08BE5F6
:1040E00090E02FE438E040C021323105E1F0223287
:1040F000310531F135C082E190E02AEA38E034C080
:1041000099278130910549F028F0029749F5E1E2BD
:10411000F8E005C0EBE4F8E002C0EDE2F8E08491DD
:1041200090E09F0121C063307105D0F4660F771FC6
:10413000FB01EB56FE4F2081318189E090E014C0F5
:104140006330710568F4FB01EE0FFF1FE157FE4F6E
:1041500020813181FB01E457FE4F808190E004C053
:1041600080E090E020E030E0FA0131832083089580
:1041700080E189BD82E189BD09B400FEFDCF809157
:10418000D8008F7D8093D8008091E000826080937A
:10419000E0008091E00081FDFCCF0895CF92DF9296
:1041A000EF92FF920F931F93CF93DF93EC018B015C
:1041B0007A010E942C22811133C0E114F10439F0FC
:1041C000F70180819181081B190BC80FD91FC12CE1
:1041D000D12C0115110519F18091E80085FD16C05B
:1041E0008091E8008E778093E800E114F10449F0B3
:1041F000F70180819181C80ED91ED182C08285E0ED
:104200000FC00E942C22882321F30AC08991809339
:10421000F10001501109FFEFCF1ADF0ADACF80E079
:10422000DF91CF911F910F91FF90EF90DF90CF9092
:1042300008952091C1023091C2022617370748F035
:104240006115710539F42091E8002E772093E8007C
:1042500001C0B901FC0120E06115710579F180917F
:10426000BA028823F1F18530F1F18091E80083FDF5
:104270003CC08091E80082FD2EC08091E80080FF64
:10428000EBCF2091F3008091F20090E0922B61152A
:10429000710551F08830910538F421912093F10097
:1042A000615071090196F3CF21E0089709F020E0F1
:1042B0008091E8008E778093E800CECF2111CFCF98
:1042C0000AC08091BA02882361F0853061F0809144
:1042D000E80083FD0AC08091E80082FFF2CF80E011
:1042E000089582E0089583E0089581E00895209183
:1042F000C1023091C2022617370748F061157105D7
:1043000039F42091E8002E772093E80001C0B9012C
:10431000FC0120E06115710591F18091BA028823BA
:1043200009F440C0853009F43FC08091E80083FD66
:104330003DC08091E80082FD2FC08091E80080FFA1
:10434000E9CF2091F3008091F20090E0922B61156B
:10435000710559F08830910540F424912093F100C3
:104360003196615071090196F2CF21E0089709F06A
:1043700020E08091E8008E778093E800CBCF211178
:10438000CCCF0AC08091BA02882361F0853061F0F9
:104390008091E80083FD0AC08091E80082FFF2CF9F
:1043A00080E0089582E0089583E0089581E0089513
:1043B000982F973068F59093E900981739F070912D
:1043C000EC002091ED005091F00003C0242F762FD7
:1043D00050E021FD02C09F5FECCF3091EB003E7FAB
:1043E0003093EB003091ED003D7F3093ED00309144
:1043F000EB0031603093EB007093EC002093ED0004
:104400005093F0002091EE0027FDE5CF80E0089565
:104410008F708093E90081E008958091BB0287FF4F
:1044200011C08091E80082FD05C08091BA0281111F
:10443000F8CF11C08091E8008B770BC08091BA0251
:10444000882349F08091E80080FFF8CF8091E80050
:104450008E778093E80008952091E4003091E50084
:1044600095E64091EC00842F817040FF23C080913D
:10447000E80080FD1DC08091BA02882399F0853044
:1044800099F08091EB0085FD11C04091E4005091BE
:10449000E5002417350729F3915011F09A01E1CF77
:1044A00084E0089582E0089583E0089581E008950E
:1044B00080E008954091E80042FFDDCF08950E941A
:1044C000CD220E94D522E0EEF0E0808181608083E1
:1044D000E8EDF0E080818F77808319BCA7EDB0E034
:1044E0008C918E7F8C9380818F7E80831092B90215
:1044F00008950F931F93CF93DF930E94CD220E94C4
:10450000D522C8EDD0E088818F7788838881806844
:10451000888388818F7D888319BC1092BA0210929B
:10452000B6021092B8021092B70200EE10E0F80145
:1045300080818B7F808388818160888342E060E016
:1045400080E00E94D821E1EEF0E080818E7F8083C0
:10455000E2EEF0E0808181608083808188608083EA
:10456000F80180818E7F8083888180618883DF91DC
:10457000CF911F910F910895E8EDF0E080818F7E3B
:104580008083E7EDF0E080818160808384E082BFFA
:1045900081E08093B9020C947922E8EDF0E080810B
:1045A0008E7F80831092E20008951092DA001092BC
:1045B000E10008951F920F920FB60F9211242F93CE
:1045C0003F934F935F936F937F938F939F93AF939B
:1045D000BF93EF93FF938091E10082FF0BC0809126
:1045E000E20082FF07C08091E1008B7F8093E100B1
:1045F0000E949D1E8091DA0080FF1FC08091D8002C
:1046000080FF1BC08091DA008E7F8093DA0080915A
:10461000D90080FF0DC080E189BD82E189BD09B468
:1046200000FEFDCF81E08093BA020E94641E05C0A7
:1046300019BC1092BA020E94761E8091E10080FFA0
:1046400019C08091E20080FF15C08091E2008E7F4A
:104650008093E2008091E20080618093E20080918B
:10466000D80080628093D80019BC85E08093BA029C
:104670000E94831E8091E10084FF30C08091E2009F
:1046800084FF2CC080E189BD82E189BD09B400FEB0
:10469000FDCF8091D8008F7D8093D8008091E1007C
:1046A0008F7E8093E1008091E2008F7E8093E20014
:1046B0008091E20081608093E2008091B6028823BD
:1046C00011F084E007C08091E30087FD02C081E023
:1046D00001C083E08093BA020E948F1E8091E100A6
:1046E00083FF29C08091E20083FF25C08091E10013
:1046F000877F8093E10082E08093BA021092B60235
:104700008091E1008E7F8093E1008091E2008E7FB6
:104710008093E2008091E20080618093E20042E0B9
:1047200060E080E00E94D8218091F0008860809352
:10473000F0000E947D1EFF91EF91BF91AF919F917C
:104740008F917F916F915F914F913F912F910F903A
:104750000FBE0F901F9018951F920F920FB60F92D9
:1047600011242F933F934F935F936F937F938F9376
:104770009F93AF93BF93CF93DF93EF93FF93C0913A
:10478000E900CF708091EC00D82FD17080FDD0E887
:104790001092E9008091F000877F8093F000789478
:1047A0000E94F0231092E9008091F00088608093CD
:1047B000F000CD2BCF70C093E900FF91EF91DF9116
:1047C000CF91BF91AF919F918F917F916F915F91A9
:1047D0004F913F912F910F900FBE0F901F90189502
:1047E0001F93CF93DF93CDB7DEB7AA970FB6F89498
:1047F000DEBF0FBECDBFEBEBF2E08091F100819305
:1048000022E0E33CF207C9F70E94F71E8091E8001E
:1048100083FF2EC18091BB029091BC02492F50E0D2
:104820004A30510508F024C1FA01EE59FF4F0C94AB
:104830007725803821F0823809F01AC108C08091AC
:10484000B7029091B802992389F082600FC08091DD
:10485000BF028F70873008F00BC18093E900809110
:10486000EB0085FB882780F91092E9009091E80021
:10487000977F9093E8008093F1001092F100D1C0EF
:10488000282F2D7F09F0F4C0882319F0823061F0C1
:10489000EFC08091BD02813009F0EAC0933009F089
:1048A00080E08093B8022EC08091BD0281112AC0A1
:1048B0008091BF028F702FEF280F263008F0D8C0EC
:1048C0008093E9002091EB0020FF1CC0933021F47D
:1048D0008091EB00806214C09091EB009061909306
:1048E000EB0021E030E0A90102C0440F551F8A957A
:1048F000E2F74093EA001092EA008091EB008860B2
:104900008093EB001092E9008091E800877F80930C
:10491000E8000E940D22ACC08111AAC01091BD0216
:104920001F778091E3008078812B8093E300809152
:10493000E800877F8093E8000E940D228091E800C4
:1049400080FFFCCF8091E30080688093E300111129
:1049500002C082E001C083E08093BA0289C080581F
:10496000823008F085C08091BD029091BE028C3DDE
:1049700053E0950779F583E08A838AE289834FB70C
:10498000F894DE01139620E03EE051E2E32FF0E0E0
:1049900050935700E49120FF03C0E295EF703F5F12
:1049A000EF708E2F90E0EA3010F0C79601C0C096ED
:1049B0008D939D932F5F243149F74FBF8091E8007D
:1049C000877F8093E8006AE270E0CE0101960E9442
:1049D000192116C06091BF027091C002AE014F5FF5
:1049E0005F4F0E946020BC01892B09F441C0909167
:1049F000E800977F9093E80089819A810E9477214F
:104A00008091E8008B778093E80032C0803881F590
:104A10008091E800877F8093E8008091B6028093C0
:104A2000F1008091E8008E7772CF811121C08091D2
:104A3000BD029091BE0299270297D4F48091E800BC
:104A4000877F8093E8008091BD028093B6020E9428
:104A50000D228091B602811106C08091E30087FD8E
:104A600002C081E001C084E08093BA020E94DE1E91
:104A70008091E80083FF0AC08091E800877F8093DF
:104A8000E8008091EB0080628093EB00AA960FB65D
:104A9000F894DEBF0FBECDBFDF91CF911F91089577
:104AA000CF938091BA028823A1F0C091E900CF7022
:104AB0009091EC00892F817090FD80E8C82B1092B6
:104AC000E9008091E80083FD0E94F023CF70C0933D
:104AD000E900CF910895991B79E004C0991F9617BA
:104AE00008F0961B881F7A95C9F780950895EE0FF8
:104AF000FF1F0590F491E02D0994FB01DC0104C037
:104B00008D910190801921F441505040C8F7881BC5
:104B1000990B0895F999FECF92BD81BDF89A992716
:104B200080B50895A8E1B0E042E050E00C94BE25C5
:104B3000262FF999FECF92BD81BDF89A019700B456
:104B4000021639F01FBA20BD0FB6F894FA9AF99AF6
:104B50000FBE08950396272F0E9499250E9498253D
:104B6000252F0E949925242F0C9499250196272FF3
:104B70000E9499250C949825DC01CB01FC01F99940
:104B8000FECF06C0F2BDE1BDF89A319600B40D9299
:0C4B900041505040B8F70895F894FFCF52
:104B9C00C8003502001E041E631E5F1E5B1E031E32
:104BAC0001E200E900EA00B500B600B700CD0083D1
:104BBC0001CC008A019201940121022302240225D6
:104BCC0002260227022A02B300B4006F0070008193
:104BDC008283E200E900EA00B500B600B700CD0020
:104BEC008301CC008A019201940121022302240248
:104BFC002502260227022A02B300B4006F007000BF
:104C0C00818283909192939594969734353667F779
:104C1C00F6F5F4F1F0C630313332376640322210FB
:0C4C2C0009DE08BC0861087A0893080043
:00000001FF
